:030000000219FDE5
:03000B000200AA46
:03002B0002015C73
:03005B000202F0AE
:030073000202DDA9
:1000800002030406080C10182030406080040608A3
:100090000C10182030406080A0C00003070F1F0D17
:1000A0000D04050D050305030302C2AFC0D0C0E077
:1000B000206214E5256009E473E525F4F58AD2622F
:1000C000D0E0D0D0D2AF3285268AC262E526F46075
:1000D0002F30682520720DD0E0D0D0C292C291C2DC
:1000E00090D2AF32C292C291C290206F0C206509AB
:1000F0007405D5E0FDE57B4290D0E0D0D0D2AF32A0
:10010000758A00C28DD26201F901B9306805206597
:1001100002D29201B9306805206502D29101B9304E
:100120006805206502D29001B9C29530680A206541
:1001300007740CD5E0FDD29201B9C29430680A2050
:100140006507740CD5E0FDD29101B9C29330680AFD
:10015000206507740CD5E0FDD29001B9C2AFC2ADE5
:1001600053E6EFC0D0C0E0D2D3D2AFC2CEE52A6012
:1001700007207449152A21BD7800790020742EE5E6
:1001800080307E01F430E70278FF53DACF207E031F
:1001900043DA20307E0343DA10C2D8C271E58030E2
:1001A0007E01F430E70279FFC3E89970CB30610338
:1001B000752A18207403752A18885CD27020740D73
:1001C000E52B6004152B21CD43DA01C2D820700243
:1001D000413CA85C206102C2702074367982B70469
:1001E00031C3E894F0400374F0F8E8C4540F28F8E1
:1001F0007984B703024112C313C313872120080275
:10020000C313200A06C3C898F8411228F850037493
:10021000FFF88822E52D54066022206B1FE536C3C7
:1002200033C333F8E564C313C313F9C39522400203
:100230008922E82522F52250037522FF7882B60430
:1002400059852224A824C3E52495614002A861C3EE
:10025000E895634002A8638825E5667002418DC376
:10026000E8AA669A5003E8FAE4F9EAC333FBE568C2
:10027000F45B29400D2567F8E56760021567400BC0
:10028000418D0AC3E5679A5002056778FF8826C248
:100290006FC3E52694F84002D26F20CF0AD0E0D099
:1002A000D043E610D2AD32C2CF053A7801E52A60DC
:1002B00005307402152AC3E55C94014005755F00A2
:1002C00041D3756000756900E55F2401F55F500357
:1002D000755FFFD0E0D0D043E610D2AD32C2AF534D
:1002E000E67F7592FA7593FFC260759104D2AF32C2
:1002F000C2AF53E6EFC2ADC0D0C0E0C0F0D2D3D29F
:10030000AFA8FBA9FCC2D8307102615753DACF20E5
:100310007E0343DA10307E0343DA20D271E5803069
:100320007E01F420E702612E88278928A18453DA10
:10033000CF207E0343DA20307E0343DA10C2D8C2D6
:1003400071307402A1707800E580307E01F430E7EE
:1003500002A170885CA15853DACF207E0343DA20D3
:10036000307E0343DA10C271206102813053DACF4C
:10037000207E0343DA10307E0343DA20C2D8D271E4
:1003800088578958C3E89555F8E99556F97B007E5A
:10039000087A00C3E8948CE994005005755B0081ED
:1003A00022882178A2E6A8216055C3E894C8E99480
:1003B000005008E4D2E4FB7A0A61FDC3E89468E9DE
:1003C00094015008E4D2E3FB7A0F61FDC3E894D0B6
:1003D000E994025008E4D2E2FB7A1E61FDC3E8947E
:1003E000A0E994055008E4D2E1FB7A3C61FDC3E842
:1003F0009498E994085008E4D2E0FB7A787E00C330
:10040000E89559FCE9955AFD30E70AECF42401FC23
:10041000EDF43400FD755B00C3EC9AED9E5003755E
:100420005B018859895A8557558558567802A158D5
:10043000C3E89527F8E99528F9307C02A13C307B88
:1004400002A13C307A02A1352075028153E9FDE812
:10045000FC8172E9C313F9E813F8307902A135E998
:10046000C313F9E813F8307802A135E9C313FDE8A6
:0E04700013FC20612CC3EC941CED940240029E
:10047E008189ED701EC3EC94C850180529E52970CA
:10048E00021529C3E529940A5002A170755C00D2A9
:10049E0070A170E529600215297888E6F9740020AC
:1004AE007F087896B90302789EE624FAFEE43400BB
:1004BE00FFC3EC9EFCED9FFD9208B90310A20850FD
:1004CE0007207609D27681DB307602C276A20850FA
:1004DE0016B9030DECF42401FCEDF43400FD020416
:1004EE00F578007900A13CB90315EC33FCED33FD32
:1004FE00C3EC940AFCED9400FD50047C007D00C317
:10050E00EC94FFED9400400678FF7900A13CEC8559
:10051E0072F0A4C5F0A2F733F87900400302055833
:10052E0078FF7900020558E9C313F9E813F8307C17
:10053E000EE9600278FFC3E81338F8E43400F9C31B
:10054E00E894FFE99400400278FF885CD270206145
:10055E0002A170741FF4552F4BF52FC274EB70026D
:10056E00D274752A18307403752A0A306102A18478
:10057E0020740353DAFE207403752B06D0F0D0E0FE
:10058E00D0D0D2AD43E6103279010205B479030220
:10059E0005B4790A0205B4791E0205B47964020520
:1005AE00B479C80205B47817E4D5E0FDD8FAD9F6C7
:1005BE00227A147B780205DB7A107B8C0205DB7ABB
:1005CE000D7BB40205DB7A0B7BC80205DBE573D528
:1005DE00E001227902E4C294D5E0FDD291D5E0FD8E
:1005EE00C291D5E0FDD294D5E0FDE920E002D29291
:1005FE0030E002D290E573D5E0FDE920E002C29230
:10060E0030E002C2907496D5E0FDD9C9EAF8D5E083
:10061E00FDD8FBDBB8C29422C37C007D0075F000D0
:10062E0005F0EA33FAEB33FB50F6EB13FBEA13FA61
:10063E00C3E9FFE8FEE89AF8E99BF95004EFF9EEFA
:10064E00F8B3EC33FCED33FDD5F0DFEDF9ECF82229
:10065E00E889F08A20D2D4F8A9F07B0030F70B7B22
:10066E00FFF42401F8E9F43400F9E88520F0A4AD94
:10067E00F0F8E98520F0A4AFF0FEED2EF974003FFE
:10068E00FA7C04C3EA13FAE913F9E813F8DCF48BE5
:10069E00F030F70AE8F42401F8E9F43400F9E889B7
:1006AE00F0C2D4F8A9F0227882B60403020710C370
:1006BE00E55C940140030206DA852224E4F544F554
:1006CE0045F546F547F548C26E0207107882E6FCFE
:1006DE00D26EE522F523783879C7AA40AB41C3EB39
:1006EE0013FBEA13FAEC146013C3EB13FBEA13FAD1
:1006FE00EC14146007C3EB13FBEA13FAD1268844FB
:10070E00894522C3E5449523F8E5459400F9500C3C
:10071E00C3E89480E994FF4016020741C3E8947F32
:10072E00E994005003020741787F7900020741786F
:10073E008079FF8849894A22E5492546F8E54A35F8
:10074E0047F9854A20E4300701F43548FA30E709C5
:10075E00C3EA94F0401502077FC3EA940F500302D8
:10076E00077F78FF79FF7A0F02077F780079007A8A
:10077E00F0C3E5249561500AC374019524500B0211
:10078E00079DE54A20E70E02079DE54A30E70688F9
:10079E004689478A482278A5E6FAC3E54933F8E543
:1007AE004A33F9D15EE930E70BC3E89480E994FF50
:1007BE004013E1D7C3E8947FE994005002E1D77863
:1007CE007F7900E1D7788079FFE820E715C3E5232C
:1007DE0098F84009C3E8940140030207FE7801022D
:1007EE0007FEE8F424012523F840030207FE78FFF4
:1007FE00884B2278A6E6FAA847A94812065EE93089
:10080E00E70CC3E89401E994FF4016020833C3E8ED
:10081E0094FFE99400500302083378FF7900020830
:10082E0033780179FFE920E715C3E54B98F84009C5
:10083E00C3E89401400302085A780102085AE8F40A
:10084E002401254BF8400302085A78FF88242278A9
:10085E00FF20692879A1E76023E541601F74FF85B9
:0E086E0041F0848539F0306A0375F005A4F876
:10087C00C5F0600278FFC3E895645002A8648863F1
:10088C0022C3E5409440E5419401E5635003140113
:10089C009E046002F563220208A62275E890227875
:1008AC0083E6FF30EDF9A8BDA9BE0570C3E57094D1
:1008BC00084052757000E9FA79A0E76044EA7007C5
:1008CC00E571601B0208DFC3E895716010E571509B
:1008DC0006600C140208EB0460F90208EBE571F5F4
:1008EC0071C3946D401B7561C0C394044013756152
:1008FC0080C39404400B756140C39404400375613C
:10090C000075BB0622E5612410500274FFF5617975
:10091C0082B704022138C3A861E524985002A824A8
:10092C00C3E895634002A86388258826E570B40760
:10093C000375BB1022743279A787F0A4C5F0A2F717
:10094C0033F8C3E895614002A86188228824882581
:10095C0088268864227540007541F022C2AF75C8A4
:10096C0020A8CCA9CDAA3A30CF010A75C824D2AFA1
:10097C00AB3BAC3C883B893CC3E89BF8E99C2069C9
:10098C0008F9306602417721D1AD3D8A3DF9EA9DE7
:10099C00FA600478FF79FFAE3EAF3F8B3E8C3FA8E8
:1009AC003BA93CC3E89EF8E99FF9C3E54113FBE57D
:1009BC004013FAE82AF540E93BF54150067540FF33
:1009CC007541FF411EAA40AB41AC40AD417E047F56
:1009DC0002C3EB9404400D1E1FC3EB94084005208A
:1009EC006A021E1FC3ED13FDEC13FCDEF7C3EA9C79
:1009FC00FAEB9DFBEF6009C3E913F9E813F8DFF795
:100A0C00EA28FAEB39FB8A408B4150067BFF8B407E
:100A1C008B41C3EB94025002D2663069047F0341D0
:100A2C00497892E6FFC3E537948240110FC3E5374E
:100A3C0094A040010FC3EF940640027F057E02E5AF
:100A4C0041C4540FF9E541C454F0F8E540C4540FC7
:100A5C0028F8C3E89EFAE99400FB4009C3EA940223
:100A6C00EB940050047A02E4FB41C3AA40AB41EB87
:100A7C00C4FEEAC4540F4EFCC3EA9CFAEB9400FB90
:100A8C00C3E813C313F8EA28FAEB3400FB8A408B53
:100A9C0041C3EB94024002C2667802EBC4FE7B00B9
:100AAC00EAC4540F4EFAC3EA98FA4005C3940250B4
:100ABC00027A027892E6FF30600241C3855192853A
:100ACC005293D26043E680C3E49AF8E49BF9306613
:100ADC0002614FE8FAE9FBD3E913FDE813FC8851F6
:100AEC008952C3EF94036038EF20E00DE82CF8E94D
:100AFC003DF9ECFAEDFB020B18E828F8E939F9C3DB
:100B0C00E82402F8E93400F97AFE7BFFC3EF940382
:100B1C00400E8A538B54884D894E8C4F8D50618377
:100B2C00885389548A4D8B4E8C4F8D503069127579
:100B3C0053F07554FF754FF07550FF7551F07552A9
:100B4C00FF6183E8FAD3E813FC8851C3EF94036088
:100B5C0020EF20E007E82CF8ECFA616FE82824027B
:100B6C00F87AFEC3EF940340088A53884D8C4F618A
:100B7C008388538A4D8C4FE568C3335002646BF500
:100B8C0068306002618D753402D26043E680E52DD9
:100B9C0054066034A840A941C3E913F9E813F8C31B
:100BAC00E913F9E813F8306904E92440F9C2AF53AA
:100BBC00E67F759100C3E498F594E499F5957591E9
:100BCC0004D26043E680D2AF22D264754300752014
:100BDC0000306C03752040020BF4D2647543007531
:100BEC002040306C0375200078017901206620E5E7
:100BFC002D54066002C2647914E541C313700104DC
:100C0C00F8C3941440027814306904781B791B20C3
:100C1C006010E543600C306903D53404D26D819FBC
:100C2C0071950543E59BF45440B5200281893069E8
:100C3C000908C3E899400118811B20640A08C3E81D
:100C4C0099400261F4811BC264C2AF53E67F759177
:100C5C00003066127594007595F8759104D2604356
:0F0C6C00E680D2AF61F4E5417EFFC3334005C39C
:100C7B00334001FEC3E49E759400F5958166C3E590
:100C8B00339401500261F430640261F4D802819D07
:100C9B00811BC26DC2AF53E67F759100855394855E
:100CAB005495759104854D92854E93D26043E680A1
:100CBB00D2AFE52D54066008206A020533020CDB27
:100CCB00306D0D206C0A2064071581158102158A81
:100CDB002278003064027801E53775F007A4F9E556
:100CEB00F028F5F0E9A2F013A2F113A2F213F537F5
:100CFB00C394785003753778C3E53795384008D2DD
:100D0B0065C292C291C290306002A112854F92854A
:100D1B005093D26043E68022207D16C2AF7542020B
:100D2B00C294D295306202D290D2AF759F11020F4E
:100D3B0012C2AF754202C294D293306202D292D2E7
:100D4B00AF759F11020F12307243207D20C2AF7519
:100D5B00420390013A757B10C290C293306204D269
:100D6B0091A170D294D2AF759F01020F12C2AF75D1
:100D7B00420390013A757B10C292C295306204D245
:100D8B0091A190D294D2AF759F21020F12207D17A3
:100D9B00C2AF754203900115C290306202D291D25C
:100DAB00AF759F01020F12C2AF754203900115C2BE
:100DBB0092306202D291D2AF759F21020F12207D29
:100DCB0016C2AF754204C295D293306202D291D251
:100DDB00AF759F21020F12C2AF754204C293D29519
:100DEB00306202D291D2AF759F01020F1230724363
:100DFB00207D20C2AF754205900129757B20C291E1
:100E0B00C294306204D292C116D295D2AF759F11A3
:100E1B00020F12C2AF75420590014B757B08C29150
:100E2B00C294306204D290C136D293D2AF759F1167
:100E3B00020F12207D17C2AF75420590010BC291B4
:100E4B00306202D292D2AF759F11020F12C2AF75F0
:100E5B00420590011FC2913062EBD290D2AF759FC9
:100E6B0011020F12207D16C2AF754206C293D294A7
:100E7B00306202D292D2AF759F01020F12C2AF75D0
:100E8B004206C295D294306202D290D2AF759F21A6
:100E9B00020F12307243207D20C2AF7542019001C8
:100EAB004B757B08C292C295306204D290C1BCD202
:100EBB0093D2AF759F21020F12C2AF754201900101
:100ECB0029757B20C290C293306204D292C1DCD2CE
:100EDB0095D2AF759F01020F12207D17C2AF7542DD
:100EEB000190011FC292306202D290D2AF759F2146
:100EFB00020F12C2AF75420190010BC29030620219
:100F0B00D292D2AF759F01C26522900109757B0009
:100F1B00C292C291C290C295C294C293C26222780D
:100F2B008076090876090876040876FF08760308A8
:100F3B0076FF08760B087603087601087601788C25
:100F4B0076010876FF0876FF0876FF0876FF0876AD
:100F5B00FF0876030876FF0876FF0876FF087625EC
:100F6B000876D00876280876500876040876FF08AD
:100F7B00760208760008767A0876FF0876010876FE
:100F8B0001087600087603087600227887E6FFC210
:100F9B0072BF0302D2727888E6C394036008C27DE5
:100FAB00E630E102D27DC27E7889E630E102D27E64
:100FBB00C3EF94026008758E01D273020FCE758E4B
:100FCB0000C273227880E6149000809378A5F6789F
:100FDB0081E6149000809378A6F67886E61490004C
:100FEB008D9378A7F67886E6F539C394025003758E
:100FFB003902789CE67538FFB402037538A0B40348
:10100B000375388278A3E61490009A93F566120F55
:10101B001522227896E6FA7897E6FB7888E6B403F1
:10102B0005C3EB940EFB307F047A007BFFC3EB9A76
:10103B00FCC3948250027C827572000572EC85723F
:10104B00F0A4C3E5F0947D40F222D27F111E12056D
:10105B00A51205A57A007B007C1012059BE55C2A86
:0F106B00FA74003BFBDCF37C04C3EB13FBEA13CA
:10107A00FADCF7FEC27F111E22757C00757D00E541
:10108A00EF20E6037520000520903FFFE52014605D
:10109A0006901DFF1460009304600375EF1453D982
:1010AA00BF7581C043FF8012059675EF0443B203F2
:1010BA00E5B3240220E70DF521E5E320E0068521CA
:1010CA00B343E301120F157580FF75A40075F19003
:1010DA0075D47F75900075A53F75F23F75D500757B
:1010EA00A60175E241120F15E4F8F6D8FD756801FC
:1010FA00120F2A1215DB78988673753001C2AF1267
:10110A0005AF1205BF1205A51205C61205A51205DF
:10111A00CD1205A5C2AF757C00757D0078FA79FA03
:10112A00308707D9FBD8F7021C00120F96120FCF8F
:10113A00111D111E78988673120F157588107589FE
:10114A000275C82475910475D84075A82275B8022D
:10115A0075E690759B80759D0075D10E75BC5875A6
:10116A00BB0675BA1175E880120596D2AF1208A3AC
:10117A0075360053DACF207E0343DA20307E0343EC
:10118A00DA1043DA01C2D8C2711205AFD2617B0309
:10119A007A0CE55B70077A0CDB0302111E1205A5B7
:1011AA0020700302111EC270E55CC3940240E1E59F
:1011BA002F541F855E5DF55EB55DD5DAD5C26153E4
:1011CA00DACF207E0343DA20307E0343DA10C2D816
:1011DA00C27178A2E67008D274E52F54E0F52FC2E6
:1011EA00757529001205AA307409C3E529940A40C5
:1011FA0002D27512059B78023074027800C3E55C4E
:10120A009840F0C2AF1205BF1205BF1205BFD2AF98
:10121A001205AF754C007888E6B403026113120513
:10122A009B788CE6C394015003021313E530C394F0
:10123A00015003021313757CA5757DF1207435C323
:10124A00E55C94FF5003021313C2AF1205D4D2AF68
:10125A001205AAC3E55C940150EFC2AF1205BF1292
:10126A0005A01205BFD2AF1205AAC3E55C94FF40E0
:10127A00E90217877F02D27F111E1205AAC2AFC2E6
:10128A007F111EAE5CC3E55C947FD2AF500261232E
:10129A00120596C2AF1205D4D2AFDFDA1155C3EEEA
:1012AA007897F61205AF12170A7F0AD27F111E121B
:1012BA0005AAC2AFC27F111EAE5CC3E55C947FD2A1
:1012CA00AF50E6120596C2AF1205BF1205A012056D
:1012DA00BFD2AFDFD61155EE24037896F6F8799788
:1012EA00E7C394824003985006E824827897F6125E
:1012FA0005AF12161D1217391205AA111EC3E55C95
:10130A0094FF50024140021787757C00757D00C327
:10131A00E55C954C4003855C4C1205AA78017988F6
:10132A00E7B403027805C3E55C9840024120C2AFE6
:10133A001205D41205D41205D4D2AF1205AF7530F6
:10134A0000E4F531F5320531E531F4703F053278C4
:10135A009AE67819146012783214600D787D146058
:10136A000878FA146003753200C3E53298401D12FA
:10137A000F15120596153275310078998673C2AF2A
:10138A001205D4D2AF789886731205AA1205A0E581
:10139A002A7005307402211E78012074027806C36F
:1013AA00E55C9840A17888E6C3940360031205AA15
:1013BA00E52A700302111EC2AF120F15E4F522F5D9
:1013CA0023F524F525F526F567D2AF7885E6C333EC
:1013DA00F565E4F544F545F546F547F548F570F544
:1013EA002CF52DF53775700875BB10120596120885
:1013FA00A730EDFDA8BDA9BEE97001F888711208F1
:10140A00AB75700875BB10120F96C2AF7561FF12EB
:10141A000941852261852262852263D2AF75220144
:10142A00752401752501752601856069756A01783B
:10143A0088E6B40307C27D307602D27DD268D269CB
:10144A00753300120E6F120E9E120961120968128C
:10145A000961120968120961120BE61206B5120C2B
:0D146A00DC120D23120968120BD5306E0341
:1014770012071120660312085D30660312088D12E9
:101487000CDC120D52120968120BE6306E031207BC
:1014970046120CDC120DC9120968120BD5306E0307
:1014A7001207A4120CDC120DF8120968120BE630B1
:1014B7006E03120801120CDC120E6F120968120873
:1014C700A7120BD5120CDC120E9E1208AB1209687C
:1014D700306932856461856462856069756A0179FE
:1014E700187A0CC3E53399400FC269D26A8A3585E9
:1014F700646185646302150CC3E55C9401400302D3
:101507001462021592306A1D206C1AE535147006B4
:10151700C26AD26B8162F535C3E55C940140030270
:10152700146202159275360078FA79A4E76002789A
:1015370003C3E55F985054307404E52A604D7888FA
:10154700E6B40317207D05207607A162307602A155
:1015570062206C07D26C85646181A178F0306C05DC
:101567008564617820C3E5419850028162306C1B25
:10157700C26CC27D307602D27DD26A75351285641F
:101587006181620536E55C6002A195753600C2AFE0
:10159700120F157887E6FE7602120F967887EEF619
:1015A700E4F522F523F524F525F526F565752C00D8
:1015B700752D00D2AF1205AA120F1578A4E66006A2
:1015C700D292D291D290307409C3E5369404400286
:1015D700211E614B901A0D782012165FE520B45535
:1015E7000CA312165FE520B4AA030215FD120F2AF9
:1015F70012161D02161C901A0378807B0A12165FBA
:10160700A308DBF9901A0F788C7B1912165FA308D1
:10161700DBF9901A2822C2AF1216A212167F901A6F
:1016270000740E121664A37407121664A3741512BD
:101637001664901A0378807B0A121663A308DBF9F5
:10164700901A0F788C7B19121663A308DBF9121610
:10165700B5121693901A2822E493F622E6438F01D7
:10166700538FFDFFC3E583941C400122EF857CB7B0
:10167700857DB7F0538FFE22438F02438F01857C10
:10168700B7857DB7901A0DF0538FFC22901A0D7411
:1016970055D164901A0E74AAD164227A3079D07821
:1016A70020901A40D15FE520F709A3DAF7227A30B4
:1016B70079D0901A40E7D16409A3DAF922AB74A86C
:1016C70075BB01027980BB02027981BB0302798273
:1016D700BB04027984BB05027986BB06027992BBFB
:1016E70007027987BB080279A3BB0902799CBB0A69
:1016F700027988BB0B027989E8F7227C051205AFCE
:10170700DCFB22C2AF1205BF1205C61205CD1205BA
:10171700D41205A01205BF1205C61205CD1205D4B5
:101727001205A01205BF1205C61205CD1205D4D2A7
:10173700AF22C2AF1205D41205CD1205C61205BFDE
:101747001205A01205D41205CD1205C61205BF1247
:1017570005A01205D41205CD1205C61205BFD2AFDA
:1017670022AE74AF75C2AF1205BF1205BF1205BF17
:101777001205A0DEF21205D41205A0DFF8D2AF22BF
:10178700F10AF102F102757401757501757600F1C0
:10179700687C05AD5C1205AFC3ED955C70F5C3E5DC
:1017A7005C9401400AC3E55C94FF40320217C3D141
:1017B700C4D11DF10AC2AF75EF14F102DCD505766D
:1017C700C3E5769403500280C6F1020575E57414EB
:1017D70090009F93F808C3E57598500280AEF10218
:1017E700F1020574C3E574940C5002809C120F2A11
:0A17F700D11DC2AF75EF14121702E6
:0319FD0002108352
:101A00000E0715090904FF03FF0B03010155AA0185
:101A1000FFFFFFFFFF03FFFFFF25D0285004FF0259
:091A2000007AFF0101000300FF40
:101A400023585037414661737423202020202020E2
:101A500023424C48454C4923463333302320202031
:101A60002020202020202020202020202020202076
:101C0000C2AFC2D353D9BF7581C043B20343FF8073
:101C1000752438752503B1DC7529A5752AF175E29F
:101C20004043F18053A47F75D4FFD2877DFA7803B7
:101C300079E67C10752200752300901DE97B0675FE
:101C400024987525013087028145208708D8FBD963
:101C5000F9DCF781B7308708D8FBD9F9DCF781B711
:101C6000B19CE493A3C39A6004DDC381B7DBDBB10D
:101C70008E6002812E7B08E493FAA3B16FDBF87AC1
:101C800030B16F752200752300B18EEAFCEBFDC305
:101C9000ED94FE400EB18E8A278B28ED30E0048A49
:101CA000828B83B18E7AC270D8C3ED94FE601950D6
:101CB000CEBD002BEC600F7520007521FF7529004B
:101CC000752A000200008100A827A9280809D80465
:101CD000D90281DCB192EA89AAF281CE0D81A3C337
:101CE000ED94035053EDA2E092007AC5C3E58294CF
:101CF00000E583941C508A200010438F02438F011B
:101D00008529B7852AB7F0300029A827A92808090E
:101D1000438F01538FFDD804D902A133C3E58394C7
:101D20001C4003A3A11689AAE28529B7852AB7F02A
:101D3000A3A116538FFC817F7AC1BD030CE493A34A
:101D4000FAB153DCF8B14B817F8181AA22AB23B178
:101D50006FEBFAEA6222752608C3E52313F523E543
:101D60002213F52250066323A0632201D526EAB18F
:101D7000DCB1DC75260AEAF4200102D287300102C8
:101D8000C287B1DCC3134002C201D526EB22B19257
:101D9000EAFB208702A192308702A197752608AE40
:101DA00024AF25C3EF13FFEE13FEB1E0B1DCC3EAAD
:101DB000133087024480FA30E703632201C3E5232E
:101DC00013F523E52213F52250066323A0632201B5
:101DD000D526D9E52265236523F52222AE24AF2539
:101DE0000E0FDEFEDFFCD20122424C48656C6934E6
:071DF000373163F3300601F7
:00000001FF
